:020000040000FA
:0400000046EF00F0D7
:080008009EB000ED18F0F2B209
:1000100025ED18F0F0B03AED18F0F2B415ED18F047
:10002000A1B21DED18F010009EB24FED18F01000B7
:10003000CD5254413A204B4552C94E59492050C1E6
:100040004C206B657061407069636E69636B2E68EC
:100050007520564F4E414C4BD6564554D52046310F
:1000600020524F424F54204D494E54412050524F40
:100070004752414D2000687474703A2F2F7777777C
:100080002E7069636E69636B2E687500EE0E806E6C
:100090000B0E826E816A110E926EC70E936EC00EA9
:1000A000946E620ED36E210ECD6E820ED56EB10EA1
:1000B000B16ED76AB36AD66AB26A0F0EBD6EBA6EF7
:1000C000070ECA6EFF0ECB6EBE6ABB6A010EC26E11
:1000D0000E0EC16E0F0EC06E036AFB6A026A2B6AB7
:1000E000216A226A296A2A6A2D6A2E6A316A050EF5
:1000F0001C6E320E0A6EFF0ECF6E800E006EFA0E70
:100100002C6EBCEC01F080A803EC03F081B4FBD7AB
:10011000828A020E0DEC03F0829A050E0DEC03F0BC
:10012000F19C81A0F17CF19A81B2F17A000EBE6E51
:10013000BB6E2BEC03F014EC03F0BCEC01F003AE4F
:1001400017EC02F06DEC02F000EC01F080EC01F035
:100150009DEF00F0F29EBE6ABB6A030E0DEC03F049
:0E01600083EF00F00B500C24E830146E1200F8
:1002000021EC02F057EC02F0046E020EFA6E0A0EB8
:100210002D18D8B4FF000450F92603D02E6A2D6A99
:0C02200012001DC01CF02E3E12002D2A02
:10030000030EFA6E1C4487EC01F0006E1200F92611
:1003100000003A0C490C620C7B0C800C850C9E0C86
:10032000B70CC60C800C800C800C800C800C800CF0
:10033000800C800C030EFA6E1C50D8901C34F926E9
:100340000000170C150C130C110C0F0C100C110CD9
:10035000120C0F0CFF00030EFA6E1C50D8901C34C8
:10036000F92600000F0C120C110C100C0F0C110CC4
:10037000130C150C170CFF00829625EC03F0C282BB
:10038000C2B2C0EF01F08286C4CF0BF0829225EC9E
:1003900003F0C282C2B2CAEF01F08282C4CF0CF075
:1003A000829025EC03F0C282C2B2D4EF01F08280C9
:1003B000C4CF0DF0809C25EC03F0C282C2B2DEEF08
:1003C00001F0808CC4CF0EF0809E25EC03F0C28239
:1003D000C2B2E8EF01F0808EC4CF0FF0809A25EC16
:1003E00003F0C282C2B2F2EF01F0808AC4CF10F0F3
:1003F000809625EC03F0C282C2B2FCEF01F0808649
:10040000C4CF11F0809425EC03F0C282C2B206EF93
:1004100002F08084C4CF12F0809225EC03F0C282F7
:10042000C2B210EF02F08082C4CF13F012000B1E94
:100430000C1E0D1E0E1E0F1E101E111E121E131E50
:100440001200266A0BC027F00C502726D8B0262AA7
:100450000D502726D8B0262A0E502726D8B0262A97
:100460000F502726D8B0262A10502726D8B0262A83
:1004700011502726D8B0262A12502726D8B0262A6F
:1004800013502726D8B0262A1C04046E0B0E042411
:10049000E96EEF501E6E275ED8A026062632273260
:1004A00026322732263227322750256E1200255059
:1004B0001E645DEF02F065EF02F00A50255CD8A0E3
:1004C000E86A1E5CD8A0020C000C0A501E5CD8A082
:1004D000E86A255CD8A0020C000C1CC01DF073EC6F
:1004E00002F01C6E12000B500C6493EF02F00B50E4
:1004F0000D64AFEF02F00B500E64C7EF02F00B502B
:100500000F64DBEF02F00B501064EBEF02F00B50C6
:100510001164F7EF02F00B501264FFEF02F00B5082
:100520001364090C010C0C500D64AFEF02F00C5079
:100530000E64C7EF02F00C500F64DBEF02F00C50BA
:100540001064EBEF02F00C501164F7EF02F00C5066
:100550001264FFEF02F00C501364090C020C0D50F2
:100560000E64C7EF02F00D500F64DBEF02F00D5088
:100570001064EBEF02F00D501164F7EF02F00D5034
:100580001264FFEF02F00D501364090C030C0E50BF
:100590000F64DBEF02F00E501064EBEF02F00E5030
:1005A0001164F7EF02F00E501264FFEF02F00E50EC
:1005B0001364090C040C0F501064EBEF02F00F50A1
:1005C0001164F7EF02F00F501264FFEF02F00F50CA
:1005D0001364090C050C10501164F7EF02F0105071
:1005E0001264FFEF02F010501364090C060C115056
:1005F0001264FFEF02F011501364090C070C125043
:100600001364090C080C1200037E827A14EC03F0C8
:1006100080A8FED714EC03F01200046E14EC03F073
:10062000042E0EEF03F01200FF0E096EFF0E086E8F
:10063000082E18EF03F0092E16EF03F01200FF0E3C
:10064000086E082E21EF03F012000F0E086E082E20
:1006500027EF03F012009E90F292F090F294A19294
:100660009E929D80F288F086F28AA082F28CF28EB1
:1006700012009D90F298F096F29AA0929D92F29CB0
:10068000F29E9E90F292F090F294A1929E92829AA3
:02069000120056
:103000009E9002A006EF18F010EF18F08188FE0ED7
:10301000CF6E00C001F001502C24CE6E022A1300A6
:103020008198F90ECF6E026A1300F29421C023F04A
:10303000FF0E216E57EF18F01300A19222C024F06A
:10304000FF0E226E81EF18F01300F29281A001D0E2
:1030500002D0829802D0828800D021C023F0D6CF3F
:1030600021F0D7CF21F0000ED76ED66EF17C57EF4E
:1030700018F01300F09081A201D002D0819A02D002
:10308000818A00D022C024F0B2CF22F0B3CF22F048
:10309000000EB36EB26EF17A81EF18F01300312A90
:1030A000280E3118D8A41300316A827A13009AECE2
:1030B00001F0286E2150285CD8A061EF18F06DEF68
:1030C00018F0829A2350215CD8A01300400EBE262F
:1030D000D8A01300FF0EBE6E13000308D8A07CEF2B
:1030E00018F0829A2150235CD8A01300400EBE5ED7
:1030F000D8B01300BE6A1300828A400EBE6E82787A
:103100001300ABEC01F0286E2250285CD8A08BEFA6
:1031100018F097EF18F0829A2450225CD8A0130080
:10312000400EBB26D8A01300FF0EBB6E1300030891
:10313000D8A0A6EF18F0829A2250245CD8A01300E1
:10314000400EBB5ED8B01300BB6A1300828A400EEB
:06315000BB6E817A130042
:020000040030CA
:0300010048100E96
:020005008080F9
:060008000FC00FE00F40E5
:00000001FF
